:020000020000FC
:0200000009C035
:040004007DC5CBC02B
:10001200C3C0F89407EF01BB08E002BB0FE304BBC7
:1000220000E005BB08E307BB07EC08BB0FE50DBF0B
:1000320004E00EBF222433244424EE24CC270FE014
:10004200F02ED1E001E0902E502EAA24AA94BB24D7
:1000520000271127B801C801D80168019801A80139
:1000620000936700009363000093650000936000B3
:100072000093610000936B000093700000936C008A
:1000820000936D0000936E0000936F0001E00093F7
:10009200660000936200009364000093690000937D
:1000A2006A0005E00093680000E009BF08E002BDB5
:1000B20004E003BF00E00FBD09E00EBD0AE00BBD86
:1000C2000AE60ABD0BE005BD0FE303BD02B5083029
:1000D200E9F708B70660076008BF01E809BF00E852
:1000E20008B900E80BBFE199FECF01E60EBBBFBA2B
:1000F200E09A0DB30F3F09F417D0E199FECF02E663
:100102000EBBBFBAE09A1DB203E3101650F009E12C
:10011200102EE199FECF02E60EBBBFBA1DBAE29ADB
:10012200E19A78948895FECF08E002BB00E005BB17
:1001320011E6E199FECF1EBBBFBAE09A0DB30030C3
:1001420039F0E199FECF1EBBBFBABDBAE29AE19A7D
:1001520012FB002705F905BB1A955AF700E005BB0B
:1001620008954394D33030F0D23121F001EF40169C
:1001720008F0D2E001E0200E3B1C06E4201601E06C
:10018200300648F022243324112D133308F019E1EC
:1001920008E5011B03BD0895BED118950FE303BD09
:1001A20040D0FA946AF40FE0F02E9DD0DADF9A94F0
:1001B20039F407E0902E5A9419F407E0502EBB242C
:1001C200A39409F4AA9404E0A01660F008E002BB2C
:1001D20000E005BB07EC08BB01E0E01629F004EBE8
:1001E20005BF04C0DBD106D004E805BF02B5083064
:1001F200E9F7189501E0501699F4092D0E7F0430A5
:1002020079F4D33068F40F2D069590FA03F906308D
:1002120038F01FE0101B012F68019801A801CC27BC
:10022200089510E001E0E01641F402E0F01628F033
:10023200F1FC03C010E1BA9A01C0BA981FBD08953B
:1002420004E0A01608F00895092F000F000F090F0F
:10025200000F080FFBE0E8E3E00FFB1D14911F3FC6
:1002620009F408950B2F000F000F0B0F000F0A0F58
:100272000C3008F00C50000F000F000F010FE19935
:10028200FECF0EBBBFBAE09A1DB31395E199FECF24
:100292000EBBBFBA1DBBE29AE19A103019F500E617
:1002A200E199FECF0EBBBFBAE09A1DB31395E19957
:1002B200FECF0EBBBFBA1DBBE29AE19A103091F499
:1002C20001E6E199FECF0EBBBFBAE09A1DB31395CA
:1002D2001F3F09F41EEFE199FECF0EBBBFBA1DBB53
:1002E200E29AE19A089563956A30E8F060E07395C6
:1002F2007630C8F070E0A4DF83958A3098F080E011
:100302009395963078F090E0A395AED0AA3010F095
:10031200A0E0B395A43030F0B23020F0A0E0B0E01D
:1003220003D04FD0D6D00895009162000395009378
:1003320062000A3038F0B0926200009163000395C7
:100342000093630049D000916300011730F144D05B
:1003520010916200101708F101E000936200B09260
:100362006300009164000395009364000A3038F042
:10037200B0926400009165000395009365000091BE
:100382006500013050F000916400033030F001E06C
:1003920000936400B092650001D008950091680056
:1003A2000395009368000A3058F0B09268000091FB
:1003B20069000395009369000A3010F0B092690059
:1003C200089500916A00039500936A00083018F0BE
:1003D20001E000936A0008950091640010916500A5
:1003E200103009F00D5FE9EFF1E0E00FFB1D099419
:1003F20009C008C00AC012C014C016C018C01AC072
:100402001CC01EC013E002E008951DD0103019F484
:1004120012E009E0089513E000E0089513E002E01D
:10042200089513E001E0089513E002E0089513E057
:1004320001E0089513E002E0089513E002E0089558
:1004420013E001E0089510916900009168001170B5
:10045200113009F40E5F11E0003029F0043019F078
:10046200083009F010E0089500916600003071F143
:1004720000916300003051F1013041F1033021F06D
:1004820000916200053010F100916A000730F1F42A
:1004920000916400033029F000916400003041F0C3
:1004A20015C0A23099F4B03089F4A3E0B0E0089509
:1004B20000916700013051F0A33041F4B03031F4C3
:1004C200A2E0B0E001E0009367000895B0926700F7
:1004D2000895009170000030E9F0013031F00330EE
:1004E20021F000916A000630A8F400916C00081710
:1004F20000916D00090700916E000A0700916F00DC
:100502000B0741F401E0E02E00917000013011F47C
:10051200B0927000089500916100003019F00A95C0
:10052200009361001091600006B3037000936000B5
:10053200101761F010916100103041F401FF03C007
:1005420000FF03C003C0E3D101C0ADD213E000FF3E
:100552001093610001FF10936100033029F01091A4
:100562006B00139510936B0010916100103011F421
:1005720010936B0010916B00143649F41DE5109333
:100582006B00003029F001FF05C000FF05C008958F
:10059200AFD20895B2D10895A8D20895CC27009180
:1005A2006A0002950695076C08BBEBEDF2E0ED0FD1
:1005B200FB1D099412C011C015C02BC034C03CC031
:1005C20044C04DC056C06AC07DC090C0ABC0B4C06C
:1005D200BCC0C4C0CCC047C16CC16B019C01AD01A1
:1005E200C3E0089506E0901670F0C0906800D090C5
:1005F2006900209164003091650040916200509141
:100602006300C1E008956B019C01AD01F3FEC3E0FC
:1006120008955FD1F2FEF1FE02C00AE0C02EC2E0F0
:10062200F2FEC1E0089555D1F2FEF1FE01C02AE0CA
:10063200C2E0F2FEC1E008954CD1F2FEF1FE01C02B
:100642003AE0C2E0F2FEC1E0089543D1F2FEF1FECB
:1006520002C04AE05AE0C2E0F2FEC1E008950AE0B8
:10066200F2FEF1FE00916600102F68019801A801C8
:10067200089540916200509163002091640030918E
:1006820065000AE0C02ED02EF2FEF1FEC090680096
:10069200F2FEF1FED0906900C1E00895409162003F
:1006A20050916300C0906800D09069002AE03AE05F
:1006B200F2FEF1FE20916400F2FEF1FE309165003F
:1006C200C1E008952091640030916500C0906800F7
:1006D200D09069004AE05AE0F2FEF1FE40916200D9
:1006E200F2FEF1FE50916300C1E008954091620074
:1006F200509163002091640030916500C0906800C1
:10070200D09069000F2D0770003051F400916A00FB
:100712000395083008F001E002950695076C08BBC6
:10072200C1E008950AE0C02ED02EF2FEF1FE6B0168
:100732009C01AD01C3E008956B012AE0392FF2FE5E
:10074200F1FE282FAD01C3E008956B013AE0282F96
:10075200F2FEF1FE392FAD01C3E008956B019C0159
:100762004AE05AE0F2FEF1FEAD01C3E00895CC2466
:10077200DD2422273327442755276624772488241B
:10078200E199FECF11E61EBBBFBAE09A8DB2E199A4
:10079200FECF10E61EBBBFBAE09A7DB21FE5E1991B
:1007A200FECF1EBBBFBAE09A0DB3600E7B1C8B1C42
:1007B2000FEF801609F48A941A958AF78694779433
:1007C200679486947794679486947794679400E408
:1007D200601602E470060FE0800640F009E0C02EC9
:1007E200D02E202F302F402F502F3CC000EA601611
:1007F20006E8700601E0800640F000EA601A06E8AA
:10080200700A01E0800A5395F1CF00E1601607E219
:10081200700600E0800640F000E1601A07E2700A0C
:1008220000E0800A4395F1CF08EE601603E07006FF
:1008320030F008EE601A03E0700A3395F5CF04E653
:10084200601600E0700630F004E6601A00E0700AFC
:100852002395F5CF0AE0601620F00AE0601AD394DF
:10086200F9CFC62C089509E1101618F419E11119EF
:1008720002C0112D1951CC24DD242227332744270D
:100882005527012F100F100F1A3018F01A50D39459
:10089200FBCFC12E09E1101618F4A601CC24DD24E9
:1008A200F2FEF1FE04C00AE01AE06801A801C2E00B
:1008B2000895062F102F68019801A801092D0295AD
:1008C2000695076C08BBFB1419F4C2E060FDC1E099
:1008D200089550917000523021F0533019F457E0CE
:1008E20001C055E0C52EDD2420916C0030916D00D1
:1008F20040916E0050916F000895D33028F0D031AE
:1009020019F0D23109F003C04424D2E108954424FD
:10091200EB1411F0EE240895E2E9F4E0ED0FFB1D73
:10092200099412C011C010C015C01DC026C02FC02E
:1009320043C04BC04CC067C084C08CC093C098C039
:100942009DC0A9C0A9C0AEC0DA9509F4D2E008E002
:10095200902E0895009170000395043008F000274E
:1009620000937000089500916C0003950A3008F01E
:10097200002700936C00ADDD089500916D00039592
:10098200063008F0002700936D00A3DD0895009162
:100992006E0010916F0003950A3010F00027139536
:1009A200123020F0043010F00027112700936E005F
:1009B20010936F008EDD089500916600039502305A
:1009C20008F000E0009366000895E8DC08950091C5
:1009D20064000395009364000A3038F0B09264001A
:1009E2000091650003950093650000916500013058
:1009F20048F000916400033028F001E000936400A5
:100A0200B092650008950091620003950093620020
:100A12000A3038F0B09262000091630003950093AF
:100A22006300DADC00916300011750F0D5DC10910D
:100A32006200101728F001E000936200B092630098
:100A4200089500916A000395083008F001E00093D0
:100A52006A0008950FE0F02E66277395763008F04D
:100A62007727089583958A3008F080E032DD089573
:100A72009395963008F090E02CDD0895A395AA3066
:100A820010F0A0E0B395A43020F0B23010F0A0E056
:100A9200B0E01FDD08950895139403E3101608F0E3
:100AA20011240895089544240E2DEE24003039F4C3
:100AB200D03131F0D13131F0DA9509F4D6E0089530
:100AC200D1E00895E199FECF02E60EBBBFBAE09AEB
:100AD2001DB3111641F0E199FECF02E60EBBBFBA7B
:100AE2001DBAE29AE19AD0E108954424DFE0089524
:100AF200D0E1EB1419F406B302FF16DB089500B33C
:100B0200AA2403FF0CC01C2D042F0295022B03FD07
:100B12001061C0FD1062086002BB15BB18951D2D47
:100B2200052F0295032B03FD1061C1FD10620860C1
:100B320002BB15BB1895FFFFFF00FFFFFFFFFFFF82
:100B420001FFFFFFFFFFFFFF02FFFFFFFFFFFF03AA
:100B5200FFFFFFFFFFFFFF04FFFFFFFFFFFF05FF98
:100B6200FFFFFFFFFFFF06FFFFFFFFFFFF07FFFF84
:020B7200FFFF83
:00000001FF
